:10000000602B82071C34363463346B3463343634EB
:100010001C34003418341C34183418341834183490
:100020007E3400343E346334603438340C34663407
:100030007F3400343E34633460343C3460346334A1
:100040003E34003438343C34363433347F34303446
:10005000783400347F34033403343F346034633401
:100060003E3400341C34063403343F346334633488
:100070003E3400347F346334303418340C340C3460
:100080000C3400343E34633463343E3463346334BC
:100090003E3400343E34633463347E346034303470
:1000A0001E3400343F34663466343E34063406343D
:1000B0000F3400340F3406340634063446346634C4
:1000C0007F340034003400340034003400341834F9
:1000D000183400346334633463346B346B347F34EA
:1000E000363400343E34633463346334633463340D
:1000F0003E340034633467346F347B347334633498
:10010000633400343C34663403340334733466346B
:100110005C3400343C344234993485348534993429
:1001200042343C343F34663466343E3436346634CC
:100130006734003463346334633463346334633466
:100140003E3400347F34463416341E34163446347C
:100150007F34003400340034003400340034003480
:10016000003400346334633463347F346334633481
:10017000633400343C34663403340334033466346B
:100180003C3400341F1CC92805161E1905129E0A8E
:100190000800CA2800000800930005100610D028A7
:1001A0001D30940000000514940BD428930BCD2827
:1001B00005340530151C0630CC20950A93001D30FF
:1001C000940005100610940BE328000006140000AC
:1001D000930BDF280530151C0430CC2008000330B9
:1001E000A0001F109E018C018D019D0150308E00DA
:1001F00050308F0010309000910020309B00FE3076
:10020000660095012114D9200529051006100C0857
:100210000A3C0319392B0D080A3C0319392B00003D
:100220001129051414301102031C00309200923081
:10023000120203189230031892001208A1188E00BF
:1002400021198F00232905149B1AD52A9B18C92A26
:100250001518C42A00001B18832A900A1008293C8C
:10026000031DCF2A1B1490031F1411080B3E0F020D
:100270000318AD2A0F08353E11020318B02A1B14CB
:100280008518062B9B14861B1B11061B1B159B1523
:1002900049291F141B19BC2A910A1108BD3C0319D6
:1002A0001B1503191F14031991030000093099004D
:1002B000990B5829000002309400861D8E03061DFC
:1002C0008E0A0E0803198E0A933C03198E03861FAB
:1002D0008F03061F8F0A0F0803198F0A933C031917
:1002E0008F03940B5D299B1D162B1B190E2B910A56
:1002F0001108BD3C03191B1503191F1403199103A1
:10030000000000001F1C8529A00B1B2B1F100330B1
:10031000A000051602309900990B8C299601323005
:100320001F239229932994290000C83093001608AE
:100330000E02051006100318612A0E08323E16023E
:1003400017140318171000000000051416080F02F8
:100350000318632A0F08323E1602971403189710E9
:10036000000011081602031C812A11080A3E160219
:10037000031C652ABB29BC29000017180614C029D4
:10038000C129273006109900990BC429C22000000A
:1003900097180614CB29CC2900000610CF29D029A4
:1003A000960A930B9729033093000000051006105E
:1003B00003309900990BDA29051406309900990B3E
:1003C000DF29061433309900990BE4290000930BC0
:1003D000D529EA290510061003309900990BEE295A
:1003E000051406309900990BF32906142E30990054
:1003F000990BF8290C089400940D940D940D0D0898
:100400009200920D920D920D052A003066009D011A
:100410009601103093000C2A051006100330990045
:10042000990B102A00000514000003309900990B65
:10043000172AC220061403309900990B1D2A1408AC
:10044000FC3E01201B1AFF3A8600860C860C860CA7
:10045000860C860C860C860C06141C309900990BB1
:100460002F2A0000120801201B1EFF3A8600860C6E
:10047000860C860C860C860C860C860C06141D18C1
:10048000940A1D18920A9D0A04309900990B462A75
:10049000930B0B2AFE306600000005100610033097
:1004A0009900990B512A051406309900990B562A88
:1004B000061432309900990B5B2A00001E301F236E
:1004C0000329622AA229642AAF29662A672A1718F3
:1004D00006141008293C9A00000010080610990024
:1004E000990B702A0614742A1A0806109900990BA1
:1004F000772A9718061400007D2A7E2A0610802A83
:10050000D029822ABA299003031DCA2A1F141B105E
:10051000900A11080B3E0E0203189E2A0E08353E63
:1005200011020318A12A1B1086180A2B9B14861986
:100530001B1106191B159B151F144A299F2AA02A57
:1005400000009B161B1EA92A8D0A1F140000A82A52
:100550004A291B160000AC2A4A29AE2AAF2A0000FD
:100560009B161B1AB82A8C0A1F140000B72A4A29A6
:100570001B120000BB2A4A29910303191B110319FE
:100580001F140319910A562916309900990BC62A8F
:100590005B292B2906309900990BCC2A4A29063071
:1005A0009900990BD12A00004A291B1AEF2A000052
:1005B000013090000E08143E910020309B00861DF3
:1005C0001B15861C9B12861C1F14A1189B12A118B8
:1005D0001F1400000F309900990BEC2A5B2928307A
:1005E00090000F08143E910031309B00861F1B15B0
:1005F000851C9B12851C1F1421199B1221191F1485
:1006000000000F309900990B032B5B29072B082B57
:1006100000005B290B2B0C2B00005B2991030319B5
:100620001B1103191F140319910A81290230990023
:10063000990B182B812900008A2910301F2B930059
:10064000212B00000510061003309900990B262B72
:10065000073005149900990B2B2B21180614C22082
:100660002F309900990B322B930B222B0000051091
:10067000F52BFF308600FE306600861C3D2BFF30D8
:100680009900990B412B21101F1000306600D920D2
:100690008E301F2300301B1A0830B2234F2B8D30B1
:1006A0001F23FF308600FE3066008618452B861C0F
:1006B000572BFF309900990B5B2B861C572B602B17
:1006C000211020309D000330A0001F109E010E302D
:1006D000650000306600D9201D231D231D23103026
:1006E000712BB2231D23742B3830B2231D231D23FD
:1006F0001D237A2B1830B2231D231D087F2BB22314
:10070000812B62301F23FF308600FE3066001D08FB
:10071000061D2030061E3030861E283006109D0033
:1007200003309900990B922B061459309900990BBC
:10073000972B8618692B861C9B2BFF309900990BF1
:100740009F2B861C9B2BA11021151D08203C0319F3
:1007500021111D08303C0319A114FF309900990B99
:10076000AF2BEF28A2009601083093000510083047
:1007700092002430840022088900BE2BBF2B000089
:100780000514831608148312080816070120800038
:10079000840A890A920BC12B0E309900990BCE2B3B
:1007A000960A051008309200243084000230990027
:1007B000990BD82B05140D309900990BDD2B0008EF
:1007C0008600860C860C860C860C860C860C860CA5
:1007D0000610840A920BDF2B08309900990BEE2B40
:1007E000930BB62B00000510F52B02309900990BE6
:1007F000F72B0000051438309900990BFD2B0800E9
:08400000FF3FFF3FFF3FFF3FC0
:02400E00E93F88
:104200005000580060000800A800680070007800A6
:104210005000580060001000A8006800700078008E
:10422000A800A8005000700078008000A800A80036
:10423000500058000800A800A800500058001000C6
:10424000A800B000A800A800A800A800B000A8001E
:10425000A800B000A800A800A800A800B800A80006
:10426000A800B800A800A800A800A800B800A800EE
:10427000880090006000800098007800A000A000F6
:00000001FF
